:0200000480007A
:100000009710000093800000171100001301810178
:1000100083A1000013B2110093B2F17F13B3F1FF7B
:1000200093B3010013B40180232031002322410047
:10003000232451002326610023287100232A8100F4
:1000400097100000938040FC17110000130101FF7E
:1000500003A40000933414001335F47F9335F4FFA8
:10006000133604009336048023208100232291005C
:100070002324A1002326B1002328C100232AD10074
:1000800097100000938080F817110000130181FC85
:1000900083A6000013B7160093B7F67F13B8F6FFD8
:1000A00093B8060013B906802320D1002322E10073
:1000B0002324F1002326010123281101232A2101F1
:1000C000971000009380C0F417110000130101FA8B
:1000D00003A9000093391900133AF97F933AF9FF05
:1000E000133B0900933B0980232021012322310186
:1000F000232441012326510123286101232A710170
:1001000097100000938000F117110000130181F790
:1001100083AB000013BC1B0093BCFB7F13BDFBFF34
:1001200093BD0B0013BE0B8023207101232281019C
:10013000232491012326A1012328B101232AC101EF
:10014000171D0000130D4DED971D0000938D0DF54B
:1001500083200D0013B0F0FF23A01D0023A20D008B
:10016000971F0000938F0FF4933010001331F07F2E
:100170009331F0FF133200009332008023A00F0070
:1001800023A21F0023A42F0023A63F0023A84F0073
:1001900023AA5F00971F0000938F4FF29330100047
:1001A00013B11000133E1100933E1E0013BF1E003A
:1001B00023A00F0023A21F0023A42F0023A6CF01FA
:1001C00023A8DF0123AAEF0117150000130585E519
:1001D00097150000938505F0370610F01306C6F258
:1001E0006306B5028326C5002320D600832685003A
:1001F0002320D600832645002320D6008326050031
:100200002320D600130505016FF09FFD370510F080
:10021000130505F223200500000000000000000087
:0402200000000000DA
:101000000000000001000000FFFFFFFFFFFFFF7F67
:10101000000000800100000000000000000000004F
:10102000FFFFFFFFFFFFFFFFFFFFFFFFFFFFFFFFD0
:10103000FFFFFFFFFFFFFFFFFFFFFFFFFFFFFFFFC0
:10104000FFFFFFFFFFFFFFFFFFFFFFFFFFFFFFFFB0
:10105000FFFFFFFFFFFFFFFFFFFFFFFFFFFFFFFFA0
:10106000FFFFFFFFFFFFFFFFFFFFFFFFFFFFFFFF90
:10107000FFFFFFFFFFFFFFFFFFFFFFFFFFFFFFFF80
:10108000FFFFFFFFFFFFFFFFFFFFFFFFFFFFFFFF70
:10109000FFFFFFFFFFFFFFFFFFFFFFFFFFFFFFFF60
:1010A000FFFFFFFFFFFFFFFFFFFFFFFFFFFFFFFF50
:1010B000FFFFFFFFFFFFFFFFFFFFFFFFFFFFFFFF40
:1010C000FFFFFFFFFFFFFFFFFFFFFFFFFFFFFFFF30
:040000058000000077
:00000001FF
